:020000040000FA
:0408000054EF09F0B8
:1008100003B26DEF05F0F2B48BEF05F09EB093EFED
:1008200005F09EB29BEF05F0F2A81AEF04F0F2B2C9
:100830001CEF04F003EF09F0CD90F2929EA026EF9A
:1008400004F00101533F26EF04F0542BAEC1B2F186
:10085000AFC1B3F1B0C1B4F1B1C1B5F1AAC1AEF14C
:10086000ABC1AFF1ACC1B0F1ADC1B1F1A6C1AAF15C
:10087000A7C1ABF1A8C1ACF1A9C1ADF1A2C1A6F16C
:10088000A3C1A7F1A4C1A8F1A5C1A9F19EC1A2F17C
:100890009FC1A3F1A0C1A4F1A1C1A5F19AC19EF18C
:1008A0009BC19FF19CC1A0F19DC1A1F196C19AF19C
:1008B00097C19BF198C19CF199C19DF1CECF96F162
:1008C000CFCF97F153C198F154C199F1CF6ACE6A55
:1008D0000101536B546B9E90CD800FBC0F8E0FBAED
:1008E00075EF04F00F8A03EF09F00F8C0FBEB1EF24
:1008F00004F096C19AF197C19BF198C19CF199C1FE
:100900009DF19AC19EF19BC19FF19CC1A0F19DC137
:10091000A1F19EC1A2F19FC1A3F1A0C1A4F1A1C107
:10092000A5F1A2C1A6F1A3C1A7F1A4C1A8F1A5C1D7
:10093000A9F1A6C1AAF1A7C1ABF1A8C1ACF1A9C1A7
:10094000ADF1AAC1AEF1ABC1AFF1ACC1B0F1ADC177
:10095000B1F1AEC1B2F1AFC1B3F1B0C1B4F1B1C147
:10096000B5F101015E6B5F6B606B616B96515E2749
:1009700097515F2398516023995161239A515E27C3
:100980009B515F239C5160239D5161239E515E27A3
:100990009F515F23A0516023A1516123A2515E2783
:1009A000A3515F23A4516023A5516123A6515E2763
:1009B000A7515F23A8516023A9516123AA515E2743
:1009C000AB515F23AC516023AD516123AE515E2723
:1009D000AF515F23B0516023B1516123B2515E2703
:1009E000B3515F23B4516023B5516123D890010105
:1009F000613360335F335E33D8900101613360331C
:100A00005F335E33D8900101613360335F335E330F
:100A100000C10CF101C10DF102C10EF103C10FF1D2
:100A200004C110F105C111F106C112F107C113F1A2
:100A300008C114F109C115F10AC116F10BC117F172
:100A400034C135F111B830EF05F00101620E046FC9
:100A5000010E056F000E066F000E076F39EF05F0EF
:100A60000101A70E046F020E056F000E066F000E47
:100A7000076F5EC100F15FC101F160C102F161C1A8
:100A800003F12EEC1FF003BF04D019BE02D019A051
:100A9000108C11A051EF05F010BA51EF05F00F8046
:100AA000108A0CC100F10DC101F10EC102F10FC19C
:100AB00003F110C104F111C105F112C106F113C116
:100AC00007F114C108F115C109F116C10AF117C1E6
:100AD0000BF135C134F103EF09F00392ABB2AB98DF
:100AE000AB88030103EE00F080517F0BE92604C0C0
:100AF000EFFF802B8151805D700BD8A48B820000AA
:100B00008051815D700BD8A48B9281518019D8B42B
:100B1000079003EF09F0F2940101453F03EF09F05C
:100B2000462B03EF09F09E900101533F03EF09F0BC
:100B3000542B03EF09F09E9213A0C5EF05F00101BD
:100B40005E6B5F6B606B616B626B636B646B656B41
:100B5000666B676B686B696B536B546BCF6ACE6A5D
:100B60000F9A0F9C0F9E0101476B486B496B4A6BB4
:100B70004B6B4C6B4D6B4E6B4F6B506B516B526BA9
:100B8000456B466BD76AD66A139011B833EF07F0FE
:100B90008BB4D2EF05F010ACD2EF05F08B84109C33
:100BA000D3EF05F08B94C3CF55F1C4CF56F1C28279
:100BB00007B43DEF06F047C14BF148C14CF149C1C4
:100BC0004DF14AC14EF15EC162F15FC163F160C196
:100BD00064F161C165F196C1B6F197C1B7F198C1F1
:100BE000B8F199C1B9F19AC1BAF19BC1BBF19CC1ED
:100BF000BCF19DC1BDF19EC1BEF19FC1BFF1A0C1BD
:100C0000C0F1A1C1C1F1A2C1C2F1A3C1C3F1A4C18C
:100C1000C4F1A5C1C5F1A6C1C6F1A7C1C7F1A8C15C
:100C2000C8F1A9C1C9F1AAC1CAF1ABC1CBF1ACC12C
:100C3000CCF1ADC1CDF1AEC1CEF1AFC1CFF1B0C1FC
:100C4000D0F1B1C1D1F1B2C1D2F1B3C1D3F1B4C1CC
:100C5000D4F1B5C1D5F1010155515B2756515C2343
:100C6000E86A5D230E2E3DEF06F05CC157F15DC1D1
:100C700058F15B6B5C6B5D6B078E0201002F03EF1D
:100C800009F03C0E006F1A50E00BE00AE86612888B
:100C900018BE02D018B4108E00C10CF101C10DF1C4
:100CA00002C10EF103C10FF104C110F105C111F130
:100CB00006C112F107C113F108C114F109C115F100
:100CC0000AC116F10BC117F134C135F101018A6770
:100CD00071EF06F08B6771EF06F08C6771EF06F02D
:100CE0008D6775EF06F0A5EF06F08EC100F18FC19C
:100CF00001F190C102F191C103F10101010E046FF4
:100D0000000E056F000E066F000E076F2EEC1FF031
:100D100000C18EF101C18FF102C190F103C191F1C7
:100D200000679AEF06F001679AEF06F002679AEF04
:100D300006F00367A5EF06F08AC18EF18BC18FF133
:100D40008CC190F18DC191F10F80D57ED5BE6DD053
:100D5000D6CF47F1D7CF48F145C149F1E86AE8CF8E
:100D60004AF119BE02D019A0108C109047C100F1B1
:100D700048C101F149C102F14AC103F101010A0E62
:100D8000046F000E056F000E066F000E076F2EEC4D
:100D90001FF003AF1080010154A7DBEF06F00F9A9C
:100DA0000F9C0F9E0101000E5E6F600E5F6F3D0E87
:100DB000606F080E616F010147BFEBEF06F04867F7
:100DC000EBEF06F04967EBEF06F04A67EBEF06F052
:100DD000F28810EF07F0F2985E6B5F6B606B616BEF
:100DE000966B976B986B996B9A6B9B6B9C6B9D6BDF
:100DF0009E6B9F6BA06BA16BA26BA36BA46BA56B8F
:100E0000A66BA76BA86BA96BAA6BAB6BAC6BAD6B3E
:100E1000AE6BAF6BB06BB16BB26BB36BB46BB56BEE
:100E2000D76AD66A0101456B466B0CC100F10DC152
:100E300001F10EC102F10FC103F110C104F111C1A2
:100E400005F112C106F113C107F114C108F115C172
:100E500009F116C10AF117C10BF135C134F103EFE5
:100E600009F003EF09F00201002F8CEF08F0D59E86
:100E7000D6CF47F1D7CF48F145C149F1E86AE8CF6D
:100E80004AF1D76AD66A0101456B466BD58E1A5076
:100E9000E00BE00AE866128818BE02D018B4108E83
:100EA00017AE1C8C00C10CF101C10DF102C10EF195
:100EB00003C10FF104C110F105C111F106C112F116
:100EC00007C113F108C114F109C115F10AC116F1E6
:100ED0000BC117F134C135F10FA0109A11B87CEF96
:100EE00007F00101620E046F010E056F000E066F20
:100EF000000E076F85EF07F00101A70E046F020EC9
:100F0000056F000E066F000E076F47C100F148C164
:100F100001F149C102F14AC103F12EEC1FF003BFF8
:100F200098EF07F019BE02D019A0108C11B00F80F5
:100F30000CC100F10DC101F10EC102F10FC103F1AD
:100F400010C104F111C105F112C106F113C107F17D
:100F500014C108F115C109F116C10AF117C10BF14D
:100F600035C134F102013C0E006F00C10CF101C12A
:100F70000DF102C10EF103C10FF104C110F105C161
:100F800011F106C112F107C113F108C114F109C131
:100F900015F10AC116F10BC117F134C135F1010188
:100FA0008A67DAEF07F08B67DAEF07F08C67DAEF22
:100FB00007F08D67DEEF07F00EEF08F08EC100F14D
:100FC0008FC101F190C102F191C103F10101010E44
:100FD000046F000E056F000E066F000E076F2EECFB
:100FE0001FF000C18EF101C18FF102C190F103C168
:100FF00091F1006703EF08F0016703EF08F0026763
:1010000003EF08F003670EEF08F08AC18EF18BC181
:101010008FF18CC190F18DC191F10F80109047C17B
:1010200000F148C101F149C102F14AC103F10101D6
:101030000A0E046F000E056F000E066F000E076F9C
:101040002EEC1FF003AF1080010154A734EF08F01D
:101050000F9A0F9C0F9E0101000E5E6F600E5F6F76
:101060003D0E606F080E616F47C100F148C101F18C
:1010700049C102F14AC103F10101140E046F050ECA
:10108000056F000E066F000E076F2EEC1FF003AF0A
:101090004DEF08F0F28872EF08F0F2985E6B5F6B2C
:1010A000606B616B966B976B986B996B9A6B9B6B94
:1010B0009C6B9D6B9E6B9F6BA06BA16BA26BA36BDC
:1010C000A46BA56BA66BA76BA86BA96BAA6BAB6B8C
:1010D000AC6BAD6BAE6BAF6BB06BB16BB26BB36B3C
:1010E000B46BB56B0CC100F10DC101F10EC102F181
:1010F0000FC103F110C104F111C105F112C106F1D4
:1011000013C107F114C108F115C109F116C10AF1A3
:1011100017C10BF135C134F18BB496EF08F010AC68
:1011200096EF08F08B84109C97EF08F08B94C3CF58
:1011300055F1C4CF56F1C28207B401EF09F047C19F
:101140004BF148C14CF149C14DF14AC14EF15EC16C
:1011500062F15FC163F160C164F161C165F196C183
:10116000B6F197C1B7F198C1B8F199C1B9F19AC177
:10117000BAF19BC1BBF19CC1BCF19DC1BDF19EC147
:10118000BEF19FC1BFF1A0C1C0F1A1C1C1F1A2C117
:10119000C2F1A3C1C3F1A4C1C4F1A5C1C5F1A6C1E7
:1011A000C6F1A7C1C7F1A8C1C8F1A9C1C9F1AAC1B7
:1011B000CAF1ABC1CBF1ACC1CCF1ADC1CDF1AEC187
:1011C000CEF1AFC1CFF1B0C1D0F1B1C1D1F1B2C157
:1011D000D2F1B3C1D3F1B4C1D4F1B5C1D5F101019C
:1011E00055515B2756515C23E86A5D230E2E01EFB3
:1011F00009F05CC157F15DC158F15B6B5C6B5D6BD5
:10120000078E03EF09F002C0E0FF005001C0D8FFD5
:101210001000A6B209EF09F00CC0A9FF0BC0A8FF8F
:10122000A69EA69CA684F29E550EA76EAA0EA76E39
:10123000A682F28EA694A6B21BEF09F00C2A120029
:10124000A96EA69EA69CA680A8500C2A1200040196
:101250002C0E826F2FEC0BF029EC20F00C5020ECC0
:1012600009F0E8CF00F10C5020EC09F0E8CF01F1D3
:1012700001AF40EF09F00101FF0E026FFF0E036F97
:10128000CCEC1FF029674CEF09F00401200E826FAF
:101290002FEC0BF051EF09F004012D0E826F2FECB3
:1012A0000BF0D6EC1DF01200306A076A0F6A106A64
:1012B000116A126A136A0F010E0EC16E860EC06E9D
:1012C000030EC26E0F01896A110E926E080E8A6EAD
:1012D000F10E936E8B6A800E946EF18E81848286FD
:1012E000FC0E20EC09F0E8CF0BF00BA011800BA254
:1012F00011820BA411840BA81188C90E20EC09F0EF
:10130000E8CF17F0CA0E20EC09F0E8CF18F0CB0EAA
:1013100020EC09F0E8CF19F0CC0E20EC09F0E8CF72
:101320001AF0CD0E20EC09F0E8CF2FF01C6A1D6AF0
:101330000E6A01015B6B5C6B5D6B576B586BF29ACD
:101340000101476B486B496B4A6B4B6B4C6B4D6BA8
:101350004E6B4F6B506B516B526B456B466BD76A44
:10136000D66A0F01280ED56EF28A9D90B00ECD6E12
:1013700001015E6B5F6B606B616B626B636B646BD7
:10138000656B666B676B686B696B536B546BCF6A8D
:10139000CE6A0F9A0F9C0F9E9D80760ECA6E9D821C
:1013A00002013C0E006FCC6A160E20EC09F0E8CF6B
:1013B00000F1170E20EC09F0E8CF01F1180E20EC37
:1013C00009F0E8CF02F1190E20EC09F0E8CF03F1A3
:1013D000010103AF06EF0AF029EC20F0160E0C6EA7
:1013E00000C10BF009EC09F0170E0C6E01C10BF0F7
:1013F00009EC09F0180E0C6E02C10BF009EC09F0B3
:10140000190E0C6E03C10BF009EC09F000C18AF152
:1014100001C18BF102C18CF103C18DF100C18EF1CC
:1014200001C18FF102C190F103C191F11A0E20ECBC
:1014300009F0E8CF00F11B0E20EC09F0E8CF01F134
:101440001C0E20EC09F0E8CF02F11D0E20EC09F093
:10145000E8CF03F1010103AF5CEF0AF029EC20F0C3
:101460001A0E0C6E00C10BF009EC09F01B0E0C6E8D
:1014700001C10BF009EC09F01C0E0C6E02C10BF05F
:1014800009EC09F01D0E0C6E03C10BF009EC09F01C
:101490001A0E20EC09F0E8CF00F11B0E20EC09F049
:1014A000E8CF01F11C0E20EC09F0E8CF02F11D0E8F
:1014B00020EC09F0E8CF03F100C192F101C193F1F2
:1014C00002C194F103C195F1240EAC6E900EAB6E87
:1014D000240EAC6E080EB86E000EB06E1F0EAF6E0E
:1014E0000401806B816B0F01900EAB6E0F019D8A22
:1014F0000301806B816BC26B8B9207900001F28EAF
:10150000F28C07B084EF1CF00FB01DEF16F010BE88
:101510001DEF16F012B81DEF16F00301805181196E
:101520007F0BD8B484EF1CF013EE00F081517F0BD9
:10153000E126812BE7CFE8FFE00BD8B484EF1CF065
:1015400023EE82F0C2513F0BD926E7CFDFFFC22B3B
:10155000DF50780AD8A484EF1CF007808EC100F118
:101560008FC101F190C102F191C103F10101040E9B
:10157000046F000E056F000E066F000E076F2EEC55
:101580001FF000AFCDEF0AF00101030E8E6F000EC9
:101590008F6F000E906F000E916F03018251720ADF
:1015A000D8B402EF16F08251520AD8B402EF16F006
:1015B0008251750AD8B402EF16F08251630AD8B48A
:1015C0003EEF19F08251690AD8B4B1EF12F082519E
:1015D0007A0AD8B4C4EF13F08251490AD8B402EFA2
:1015E00012F08251500AD8B420EF11F08251700AE3
:1015F000D8B463EF11F08251540AD8B48EEF11F0D1
:101600008251740AD8B4D4EF11F08251410AD8B48F
:1016100045EF0CF082514B0AD8B443EF0BF08251E6
:101620006D0AD8B478EF10F082514D0AD8B491EF1A
:1016300010F08251730AD8B432EF15F08251530A78
:10164000D8B497EF15F08251660AD8B463EF12F060
:101650008251590AD8B4C9EF0FF075EF19F004019F
:1016600014EE00F080517F0BE12682C4E7FF802B4F
:10167000120004010D0E826F2FEC0BF00A0E826F28
:101680002FEC0BF0120004014B0E826F2FEC0BF0CD
:1016900004012C0E826F2FEC0BF081B802D02FB614
:1016A00030D003018351430AD8B488EF0BF0030113
:1016B0008351630AD8B48AEF0BF003018351520AB5
:1016C000D8B48CEF0BF003018351720AD8B48EEFBB
:1016D0000BF003018351470AD8B490EF0BF00301DC
:1016E0008351670AD8B492EF0BF003018351540A77
:1016F000D8B494EF0BF003018351740AD8B403EF0C
:101700000CF003018351550AD8B496EF0BF082D048
:101710002F807AD02F9078D02F8276D02F9274D0CD
:101720002F8472D02F9470D02F866ED084C330F166
:1017300085C331F186C332F187C333F10101296BCF
:1017400077EC20F0EEEC1FF000C104F101C105F1CF
:1017500002C106F103C107F16AEC20F0200EF86E19
:10176000F76AF66A0900F5CF2CF10900F5CF2DF1E3
:101770000900F5CF2EF10900F5CF2FF10900F5CFC3
:1017800030F10900F5CF31F10900F5CF32F1090050
:10179000F5CF33F10101296B77EC20F0EEEC1FF06F
:1017A0002EEC1FF00067DCEF0BF00167DCEF0BF0B5
:1017B0000267DCEF0BF0036701D025D004014E0E69
:1017C000826F2FEC0BF004016F0E826F2FEC0BF089
:1017D00004014D0E826F2FEC0BF00401610E826F3D
:1017E0002FEC0BF00401740E826F2FEC0BF0040150
:1017F000630E826F2FEC0BF00401680E826F2FECEA
:101800000BF073EF19F02F96CD0E0C6E2FC00BF06E
:1018100009EC09F0CD0E20EC09F0E8CF2FF02FB045
:1018200006D00401630E826F2FEC0BF005D004018B
:10183000430E826F2FEC0BF02FB206D00401720E14
:10184000826F2FEC0BF005D00401520E826F2FEC4B
:101850000BF02FB406D00401670E826F2FEC0BF053
:1018600005D00401470E826F2FEC0BF02FB606D087
:101870000401740E826F2FEC0BF005D00401540E9E
:10188000826F2FEC0BF073EF19F00401410E826FA1
:101890002FEC0BF003018351310AD8B4E9EF0EF0BD
:1018A00003018351320AD8B419EF0EF003018351BA
:1018B000330AD8B4A2EF0DF003018351340AD8B42F
:1018C00092EF0CF003018351350AD8B46FEF0CF09E
:1018D00004013F0E826F2FEC0BF073EF19F004013F
:1018E0002C0E826F2FEC0BF003018451300AD8B418
:1018F00082EF0CF003018451310AD8B48AEF0CF066
:10190000DBEF0DF08B900401300E826F2FEC0BF0AB
:1019100090EF0CF08B800401310E826F2FEC0BF0F6
:1019200073EF19F0CC0E20EC09F0E8CF0BF00401B6
:101930002C0E826F2FEC0BF003018451310AD8B4C6
:10194000B6EF0CF003018451300AD8B4B8EF0CF0B4
:10195000030184514D0AD8B4C2EF0CF00301845145
:10196000540AD8B4C9EF0CF0E0EF0CF08A8401D02F
:101970008A940BAE04D00BAC02D00BBA21D0E00E8F
:101980000B1218D01F0E0B168539E844E00B0B1212
:1019900011D0E00E0B166AEC20F085C332F186C33D
:1019A00033F10101296B77EC20F0EEEC1FF00051D0
:1019B0001F0B0B12CC0E0C6E0BC00BF009EC09F0D8
:1019C0000401340E826F2FEC0BF004012C0E826F99
:1019D0002FEC0BF0CC0E20EC09F0E8CF1AF08AB413
:1019E00006D00401300E826F2FEC0BF005D00401FD
:1019F000310E826F2FEC0BF004012C0E826F2FEC56
:101A00000BF01A38E840070BE8CF82F40401300EDF
:101A100082272FEC0BF004012C0E826F2FEC0BF0C1
:101A200029EC20F01A501F0BE8CF00F1CCEC1FF08E
:101A300032C182F40401300E82272FEC0BF033C147
:101A400082F40401300E82272FEC0BF004012C0EDF
:101A5000826F2FEC0BF029EC20F02DC000F100AFCD
:101A60000BD0FF0E016FFF0E026FFF0E036F04011C
:101A70002D0E826F2FEC0BF0CCEC1FF031C182F4F5
:101A80000401300E82272FEC0BF032C182F40401E6
:101A9000300E82272FEC0BF033C182F40401300E9C
:101AA00082272FEC0BF004012C0E826F2FEC0BF031
:101AB00029EC20F02CC000F1CCEC1FF031C182F4F5
:101AC0000401300E82272FEC0BF032C182F40401A6
:101AD000300E82272FEC0BF033C182F40401300E5C
:101AE00082272FEC0BF004012C0E826F2FEC0BF0F1
:101AF00029EC20F02EC000F100AF0BD0FF0E016FDB
:101B0000FF0E026FFF0E036F04012D0E826F2FEC8C
:101B10000BF0CCEC1FF031C182F40401300E8227AF
:101B20002FEC0BF032C182F40401300E82272FEC2F
:101B30000BF033C182F40401300E82272FEC0BF03E
:101B400073EF19F0CB0E20EC09F0E8CF0BF0040195
:101B50002C0E826F2FEC0BF003018451450AD8B490
:101B6000C6EF0DF003018451440AD8B4C9EF0DF05B
:101B700003018451300AD8B4CCEF0DF00301845135
:101B8000310AD8B4D0EF0DF0DBEF0DF00B9ED5EF9E
:101B90000DF00B8ED5EF0DF0FC0E0B16D5EF0DF002
:101BA000FC0E0B160B80D5EF0DF0CB0E0C6E0BC0A0
:101BB0000BF009EC09F00401330E826F2FEC0BF0EF
:101BC00004012C0E826F2FEC0BF0CB0E20EC09F0F1
:101BD000E8CF19F019BEF4EF0DF00401450E826F45
:101BE0002FEC0BF0F9EF0DF00401440E826F2FEC97
:101BF0000BF004012C0E826F2FEC0BF00401300E61
:101C0000826F2FEC0BF004012C0E826F2FEC0BF087
:101C100019B012EF0EF00401300E826F2FEC0BF0B2
:101C200017EF0EF00401310E826F2FEC0BF073EF03
:101C300019F0CA0E20EC09F0E8CF0BF004012C0ECD
:101C4000826F2FEC0BF003018451450AD8B455EF95
:101C50000EF003018451440AD8B458EF0EF003018A
:101C600084514D0AD8B461EF0EF003018451410A4A
:101C7000D8B45BEF0EF003018451460AD8B45EEF8E
:101C80000EF003018451560AD8B469EF0EF0030137
:101C90008451500AD8B474EF0EF003018451520AF3
:101CA000D8B477EF0EF080EF0EF00B9E7AEF0EF0C7
:101CB0000B8E7AEF0EF00B9C7AEF0EF00B8C7AEF16
:101CC0000EF0FC0E0B1685C3E8FF030B0B127AEF28
:101CD0000EF0C70E0B1685C3E8FF070BE846E84673
:101CE000E8460B127AEF0EF00B847AEF0EF00B94AD
:101CF0007AEF0EF0CA0E0C6E0BC00BF009EC09F077
:101D0000CA0E20EC09F0E8CF18F00401320E826F01
:101D10002FEC0BF004012C0E826F2FEC0BF018BE91
:101D200099EF0EF00401450E826F2FEC0BF09EEF41
:101D30000EF00401440E826F2FEC0BF004012C0E08
:101D4000826F2FEC0BF018C0E8FF030BE8CF82F492
:101D50000401300E82272FEC0BF004012C0E826F51
:101D60002FEC0BF018BCBCEF0EF00401410E826F9B
:101D70002FEC0BF0C1EF0EF00401460E826F2FEC3A
:101D80000BF004012C0E826F2FEC0BF018C0E8FF53
:101D9000380BE842E842E842E8CF82F40401300E12
:101DA00082272FEC0BF004012C0E826F2FEC0BF02E
:101DB00018B4E2EF0EF00401520E826F2FEC0BF01C
:101DC000E7EF0EF00401500E826F2FEC0BF073EF73
:101DD00019F0C90E20EC09F0E8CF0BF004012C0E2D
:101DE000826F2FEC0BF003018451450AD8B407EF42
:101DF0000FF003018451440AD8B40AEF0FF0030135
:101E000084514D0AD8B40DEF0FF01BEF0FF00B9E6D
:101E100015EF0FF00B8E15EF0FF0F80E0B1685C3B4
:101E2000E8FF070B0B1215EF0FF0C90E0C6E0BC07D
:101E30000BF009EC09F00401310E826F2FEC0BF06E
:101E400004012C0E826F2FEC0BF0C90E20EC09F070
:101E5000E8CF17F017BE06D00401450E826F2FECB5
:101E60000BF005D00401440E826F2FEC0BF004013F
:101E70002C0E826F2FEC0BF017C0E8FF070BE8CF9A
:101E800082F40401300E82272FEC0BF004012C0E9B
:101E9000826F2FEC0BF0078029EC20F028C0E8FFC0
:101EA000003B00430043030BCCEC1FF033C182F432
:101EB0000401300E82272FEC0BF004012C0E826FF0
:101EC0002FEC0BF029EC20F028C001F1019F019DBF
:101ED00029C000F10101CCEC1FF02FC182F40401F4
:101EE000300E82272FEC0BF030C182F40401300E4B
:101EF00082272FEC0BF031C182F40401300E8227CF
:101F00002FEC0BF032C182F40401300E82272FEC4B
:101F10000BF033C182F40401300E82272FEC0BF05A
:101F200004012C0E826F2FEC0BF029EC20F02AC05C
:101F300001F12BC000F1D89001330033D890013368
:101F400000330101CCEC1FF02FC182F40401300EEC
:101F500082272FEC0BF030C182F40401300E82276F
:101F60002FEC0BF031C182F40401300E82272FECEC
:101F70000BF032C182F40401300E82272FEC0BF0FB
:101F800033C182F40401300E82272FEC0BF073EF83
:101F900019F0FC0E20EC09F0E8CF0BF0030183519F
:101FA000520AD8B400EF10F003018351720AD8B47A
:101FB00003EF10F003018351500AD8B406EF10F07C
:101FC00003018351700AD8B409EF10F00301835163
:101FD000550AD8B40CEF10F003018351750AD8B438
:101FE0000FEF10F003018351430AD8B418EF10F03B
:101FF00003018351630AD8B41BEF10F024EF10F0F3
:102000000B901EEF10F00B801EEF10F00B921EEFE6
:1020100010F00B821EEF10F00B941EEF10F00B84EB
:102020001EEF10F00B961EEF10F00B861EEF10F057
:102030000B981EEF10F00B881EEF10F0FC0E0C6ECC
:102040000BC00BF009EC09F00401590E826F2FEC64
:102050000BF01190119211941198FC0E20EC09F0E4
:10206000E8CF0BF00BA011800BA211820BA41184FE
:102070000BA8118811A044EF10F00401520E826FDA
:102080002FEC0BF049EF10F00401720E826F2FEC71
:102090000BF011A853EF10F00401430E826F2FECE8
:1020A0000BF058EF10F00401630E826F2FEC0BF071
:1020B00011A262EF10F00401500E826F2FEC0BF0B2
:1020C00067EF10F00401700E826F2FEC0BF011A47B
:1020D00071EF10F00401550E826F2FEC0BF076EFCC
:1020E00010F00401750E826F2FEC0BF073EF19F0F6
:1020F00004016D0E826F2FEC0BF003018351300A47
:10210000D8B4D0EF10F003018351310AD8B4E3EF13
:1021100010F003018351320AD8B4F6EF10F075EFD6
:1021200019F004014D0E826F2FEC0BF06AEC20F0D9
:1021300084C331F185C332F186C333F10101296BC8
:1021400077EC20F0EEEC1FF003018351300AD8B495
:10215000B8EF10F003018351310AD8B4C0EF10F08A
:1021600003018351320AD8B4C8EF10F075EF19F0AB
:10217000FD0E0C6E00C10BF009EC09F0D0EF10F071
:10218000FE0E0C6E00C10BF009EC09F0E3EF10F04D
:10219000FF0E0C6E00C10BF009EC09F0F6EF10F029
:1021A0000401300E826F2FEC0BF004012C0E826FB5
:1021B0002FEC0BF029EC20F0FD0E20EC09F0E8CF1D
:1021C00000F107EF11F00401310E826F2FEC0BF0DC
:1021D00004012C0E826F2FEC0BF029EC20F0FE0E88
:1021E00020EC09F0E8CF00F107EF11F00401320E06
:1021F000826F2FEC0BF029EC20F004012C0E826F83
:102200002FEC0BF0FF0E20EC09F0E8CF00F1CCEC46
:102210001FF031C182F40401300E82272FEC0BF045
:1022200032C182F40401300E82272FEC0BF033C14F
:1022300082F40401300E82272FEC0BF073EF19F0BB
:1022400083C32AF184C32BF185C32CF186C32DF1FE
:1022500087C32EF188C32FF189C330F18AC331F1CE
:102260008BC332F18CC333F1010177EC20F0EEEC3B
:102270001FF0160E0C6E00C10BF009EC09F0170EE2
:102280000C6E01C10BF009EC09F0180E0C6E02C1C6
:102290000BF009EC09F0190E0C6E03C10BF009EC00
:1022A00009F000C18AF101C18BF102C18CF103C1B7
:1022B0008DF100C18EF101C18FF102C190F103C116
:1022C00091F102EF12F083C32AF184C32BF185C38D
:1022D0002CF186C32DF187C32EF188C32FF189C35A
:1022E00030F18AC331F18BC332F18CC333F1010178
:1022F00077EC20F0EEEC1FF000C18AF101C18BF108
:1023000002C18CF103C18DF100C18EF101C18FF1C9
:1023100002C190F103C191F102EF12F083C32AF1DF
:1023200084C32BF185C32CF186C32DF187C32EF115
:1023300088C32FF189C330F18AC331F18CC332F1E4
:102340008DC333F1010177EC20F0EEEC1FF00101B9
:10235000000E046F000E056F010E066F000E076F72
:102360003FEC1FF01A0E0C6E00C10BF009EC09F0E7
:102370001B0E0C6E01C10BF009EC09F01C0E0C6E6B
:1023800002C10BF009EC09F01D0E0C6E03C10BF03D
:1023900009EC09F000C192F101C193F102C194F17D
:1023A00003C195F102EF12F083C32AF184C32BF12C
:1023B00085C32CF186C32DF187C32EF188C32FF17D
:1023C00089C330F18AC331F18CC332F18DC333F14B
:1023D000010177EC20F0EEEC1FF00101000E046F1C
:1023E000000E056F010E066F000E076F3FEC1FF029
:1023F00000C192F101C193F102C194F103C195F1C1
:1024000002EF12F0160E20EC09F0E8CF00F1170EE3
:1024100020EC09F0E8CF01F1180E20EC09F0E8CF2C
:1024200002F1190E20EC09F0E8CF03F1CCEC1FF01B
:102430008FEC1DF00401730E826F2FEC0BF0040182
:102440002C0E826F2FEC0BF08AC100F18BC101F1D1
:102450008CC102F18DC103F1CCEC1FF08FEC1DF0AB
:102460000401730E826F2FEC0BF004012C0E826FAF
:102470002FEC0BF01A0E20EC09F0E8CF00F11B0E48
:1024800020EC09F0E8CF01F11C0E20EC09F0E8CFB8
:1024900002F11D0E20EC09F0E8CF03F190EC19F0E9
:1024A00004012C0E826F2FEC0BF092C100F193C14E
:1024B00001F194C102F195C103F190EC19F039ECEE
:1024C0000BF075EF19F00401660E826F2FEC0BF024
:1024D00003018351780AD8B484EF12F0030183B169
:1024E00002D0829601D0828683B302D0819401D03B
:1024F000818484B102D0829A01D0828A84B302D0CE
:10250000829801D08288138088EC12F073EF19F062
:1025100004012C0E826F2FEC0BF0300E82B602D02D
:10252000E89001D0E88081B402D0E89201D0E8823E
:10253000E8CF82F42FEC0BF004012C0E826F2FEC0D
:102540000BF0300E82BA02D0E89001D0E88082B859
:1025500002D0E89201D0E882E8CF82F42FEC0BF0B1
:1025600012000401690E826F2FEC0BF004012C0E97
:10257000826F2FEC0BF00101040E006F000E016F53
:10258000000E026F000E036FCCEC1FF02CC182F422
:102590000401300E82272FEC0BF02DC182F40401D0
:1025A000300E82272FEC0BF02EC182F40401300E86
:1025B00082272FEC0BF02FC182F40401300E82270A
:1025C0002FEC0BF030C182F40401300E82272FEC87
:1025D0000BF031C182F40401300E82272FEC0BF096
:1025E00032C182F40401300E82272FEC0BF033C18C
:1025F00082F40401300E82272FEC0BF004012C0E24
:10260000826F2FEC0BF00101040E006F000E016FC2
:10261000000E026F000E036FCCEC1FF02CC182F491
:102620000401300E82272FEC0BF02DC182F404013F
:10263000300E82272FEC0BF02EC182F40401300EF5
:1026400082272FEC0BF02FC182F40401300E822779
:102650002FEC0BF030C182F40401300E82272FECF6
:102660000BF031C182F40401300E82272FEC0BF005
:1026700032C182F40401300E82272FEC0BF033C1FB
:1026800082F40401300E82272FEC0BF004012C0E93
:10269000826F2FEC0BF00101340E006F000E016F02
:1026A000000E026F000E036FCCEC1FF02CC182F401
:1026B0000401300E82272FEC0BF02DC182F40401AF
:1026C000300E82272FEC0BF02EC182F40401300E65
:1026D00082272FEC0BF02FC182F40401300E8227E9
:1026E0002FEC0BF030C182F40401300E82272FEC66
:1026F0000BF031C182F40401300E82272FEC0BF075
:1027000032C182F40401300E82272FEC0BF033C16A
:1027100082F40401300E82272FEC0BF004012C0E02
:10272000826F2FEC0BF0200EF86EF76AF66A040148
:102730000900F5CF82F42FEC0BF00900F5CF82F4FD
:102740002FEC0BF00900F5CF82F42FEC0BF0090011
:10275000F5CF82F42FEC0BF00900F5CF82F42FECCB
:102760000BF00900F5CF82F42FEC0BF00900F5CF48
:1027700082F42FEC0BF00900F5CF82F42FEC0BF074
:1027800039EC0BF075EF19F08351630AD8A473EF9D
:1027900019F08451610AD8A473EF19F085516C0ABD
:1027A000D8A473EF19F08651410A3FE08651440ADC
:1027B0001BE08651420AD8B428EF14F08651350A3E
:1027C000D8B4FFEF1AF08651360AD8B454EF1BF094
:1027D0008651370AD8B4BDEF1BF08651380AD8B4F9
:1027E0001BEF1CF073EF19F00798079A04017A0E9B
:1027F000826F2FEC0BF00401780E826F2FEC0BF040
:102800000401640E826F2FEC0BF00401550E826FF1
:102810002FEC0BF011EF14F004014C0E826F2FEC33
:102820000BF039EC0BF075EF19F00788079A0401EB
:102830007A0E826F2FEC0BF00401410E826F2FECA9
:102840000BF00401610E826F2FEC0BF005EF14F01A
:102850000798078A04017A0E826F2FEC0BF00401AF
:10286000420E826F2FEC0BF00401610E826F2FEC91
:102870000BF005EF14F00101666746EF14F067678F
:1028800046EF14F0686746EF14F0696715D04F679C
:1028900051EF14F0506751EF14F0516751EF14F0FD
:1028A00052670AD00101000E006F000E016F000E8A
:1028B000026F000E036F120011B80AD00101620E00
:1028C000046F010E056F000E066F000E076F09D032
:1028D0000101A70E046F020E056F000E066F000EB9
:1028E000076F66C100F167C101F168C102F169C1FA
:1028F00003F12EEC1FF003BFEEEF14F0119A119CC0
:102900000101000E046FA80E056F550E066F020E32
:10291000076F66C100F167C101F168C102F169C1C9
:1029200003F166C186F167C187F168C188F169C1A9
:1029300089F12EEC1FF003BF0BD00101000E866F52
:10294000A80E876F550E886F020E896F118A119C31
:102950000E0E20EC09F0E8CF18F10F0E20EC09F074
:10296000E8CF19F1100E20EC09F0E8CF1AF1110EA2
:1029700020EC09F0E8CF1BF177EC1EF086C104F1E2
:1029800087C105F188C106F189C107F12EEC1FF05E
:1029900007823BEC1EF077EC1EF007923BEC1EF03A
:1029A00086C100F187C101F188C102F189C103F13B
:1029B00007923BEC1EF0CC0E046FE00E056F870E05
:1029C000066F050E076F2EEC1FF000C118F101C154
:1029D00019F102C11AF103C11BF13BD0119C119AEC
:1029E0000101800E006F1A0E016F060E026F000EBD
:1029F000036F4FC104F150C105F151C106F152C13D
:102A000007F12EEC1FF003AF05D029EC20F0118C5C
:102A1000119A12000E0E20EC09F0E8CF18F10F0EFB
:102A200020EC09F0E8CF19F1100E20EC09F0E8CF06
:102A30001AF1110E20EC09F0E8CF1BF14FC100F1A3
:102A400050C101F151C102F152C103F107823BECC7
:102A50001EF018C100F119C101F11AC102F11BC128
:102A600003F112000401730E826F2FEC0BF00401CE
:102A70002C0E826F2FEC0BF0078462C166F163C1EC
:102A800067F164C168F165C169F14BC14FF14CC197
:102A900050F14DC151F14EC152F157C159F158C1D8
:102AA0005AF1079458EC15F039EC0BF075EF19F06A
:102AB00066C100F167C101F168C102F169C103F1AA
:102AC0000101CCEC1FF08FEC1DF00401630E826F4E
:102AD0002FEC0BF004012C0E826F2FEC0BF04FC18A
:102AE00000F150C101F151C102F152C103F10101E4
:102AF000CCEC1FF08FEC1DF00401660E826F2FEC02
:102B00000BF004012C0E826F2FEC0BF029EC20F05F
:102B100059C100F15AC101F10101CCEC1FF08FEC59
:102B20001DF00401740E826F2FEC0BF01200108266
:102B30000401530E826F2FEC0BF004012C0E826FF8
:102B40002FEC0BF083C32AF184C32BF185C32CF146
:102B500086C32DF187C32EF188C32FF189C330F1CD
:102B60008AC331F18BC332F18CC333F1010177ECAD
:102B700020F0EEEC1FF000C166F101C167F102C167
:102B800068F103C169F18EC32AF18FC32BF190C3A1
:102B90002CF191C32DF192C32EF193C32FF194C365
:102BA00030F195C331F196C332F197C333F101018E
:102BB00077EC20F0EEEC1FF000C14FF101C150F1B5
:102BC00002C151F103C152F16AEC20F099C32FF117
:102BD0009AC330F19BC331F19CC332F19DC333F1F1
:102BE000010177EC20F0EEEC1FF000C159F101C1BA
:102BF0005AF158EC15F004012C0E826F2FEC0BF0FB
:102C000011EF16F0118E19A002D019AE108C18BE5B
:102C100002D018A4108E8251520A02E10F8201D014
:102C20000F928251750A02E1108401D010948251F2
:102C3000550A02E1108601D0109611A003D011A40C
:102C400001D01084078410B27FEF16F010A46BEF50
:102C500016F0B6C166F1B7C167F1B8C168F1B9C184
:102C600069F1BAC16AF1BBC16BF1BCC16CF1BDC104
:102C70006DF1BEC16EF1BFC16FF1C0C170F1C1C1D4
:102C800071F1C2C172F1C3C173F1C4C174F1C5C1A4
:102C900075F1C6C176F1C7C177F1C8C178F1C9C174
:102CA00079F1CAC17AF1CBC17BF1CCC17CF1CDC144
:102CB0007DF1CEC17EF1CFC17FF1D0C180F1D1C114
:102CC00081F1D2C182F1D3C183F1D4C184F1D5C1E4
:102CD00085F173EF16F062C166F163C167F164C1FB
:102CE00068F165C169F14BC14FF14CC150F14DC163
:102CF00051F14EC152F157C159F158C15AF10794DF
:102D00000FA0A1EF16F0010192678EEF16F0936706
:102D10008EEF16F094678EEF16F0956792EF16F02F
:102D2000A1EF16F03BEC14F092C104F193C105F150
:102D300094C106F195C107F12EEC1FF003BF3BEFE4
:102D400019F03BEC14F00101000E046F000E056F4A
:102D5000010E066F000E076F5FEC1FF011A02CD064
:102D600011A22AD0CCEC1FF0296701D007D00401B2
:102D70002D0E826F2FEC0BF039EF19F030C182F479
:102D80000401300E82272FEC0BF031C182F40401D4
:102D9000300E82272FEC0BF032C182F40401300E8A
:102DA00082272FEC0BF033C182F40401300E82270E
:102DB0002FEC0BF039EF19F012A8C5D012981AC0F9
:102DC0001BF01B3A1B42070E1B1600011B50000A8A
:102DD000D8B46FEF17F000011B50010AD8B4FBEF15
:102DE00016F000011B50020AD8B4F9EF16F0A1EF5B
:102DF00017F0A1EF17F029EC20F02AC001F12BC049
:102E000000F1D89001330033D89001330033010131
:102E1000630E046F000E056F000E066F000E076F45
:102E20005FEC1FF0280E046F000E056F000E066F9A
:102E3000000E076F2EEC1FF000C12DF029EC20F0E2
:102E400028C001F1019F019D29C000F10101A40EDC
:102E5000046F000E056F000E066F000E076F5FEC2B
:102E60001FF000C12CF000C104F101C105F102C145
:102E700006F103C107F1640E006F000E016F000E32
:102E8000026F000E036F2EEC1FF0050E046F000E94
:102E9000056F000E066F000E076F5FEC1FF000C19C
:102EA00004F101C105F102C106F103C107F129ECEA
:102EB00020F02DC000F12EEC1FF000C12EF02EC02E
:102EC000E8FF050F2D5C03E78A84A1EF17F02EC001
:102ED000E8FF0A0F2D5C01E68A94A1EF17F000C10C
:102EE00024F101C125F102C126F103C127F129EC2A
:102EF00020F02FEC20F01A501F0BE8CF00F1010159
:102F0000640E046F000E056F000E066F000E076F53
:102F10003FEC1FF024C104F125C105F126C106F1E3
:102F200027C107F12EEC1FF003BF02D08A9401D015
:102F30008A8424C100F125C101F126C102F127C113
:102F400003F13BEF19F000C124F101C125F102C1E9
:102F500026F103C127F110AE4DD0109E00C108F13B
:102F600001C109F102C10AF103C10BF1CCEC1FF060
:102F700030C1D6F131C1D7F132C1D8F133C1D9F165
:102F800008C100F109C101F10AC102F10BC103F14D
:102F900001016C0E046F070E056F000E066F000E28
:102FA000076F2EEC1FF003BF04D00101550EDA6F3E
:102FB0001CD008C100F109C101F10AC102F10BC125
:102FC00003F10101A40E046F060E056F000E066FDB
:102FD000000E076F2EEC1FF003BF04D001017F0E1F
:102FE000DA6F03D00101FF0EDA6F1C8E11AE3BEFDA
:102FF00019F0119E24C100F125C101F126C102F191
:1030000027C103F110A40CEF18F00401750E826FB4
:103010002FEC0BF011EF18F00401720E826F2FEC01
:103020000BF004012C0E826F2FEC0BF0CCEC1FF098
:10303000296720EF18F00401200E826F23EF18F0AB
:1030400004012D0E826F2FEC0BF030C182F40401CD
:10305000300E82272FEC0BF031C182F40401300EC8
:1030600082272FEC0BF004012E0E826F2FEC0BF059
:1030700032C182F40401300E82272FEC0BF033C1F1
:1030800082F40401300E82272FEC0BF004016D0E48
:10309000826F2FEC0BF004012C0E826F2FEC0BF0E3
:1030A0004FC100F150C101F151C102F152C103F110
:1030B0000101CCEC1FF08FEC1DF00401480E826F73
:1030C0002FEC0BF004017A0E826F2FEC0BF0040151
:1030D0002C0E826F2FEC0BF066C100F167C101F17D
:1030E00068C102F169C103F10101CCEC1FF08FEC62
:1030F0001DF00401630E826F2FEC0BF004012C0E07
:10310000826F2FEC0BF066C100F167C101F168C15D
:1031100002F169C103F101010A0E046F000E056F8F
:10312000000E066F000E076F3FEC1FF0000E046FDD
:10313000120E056F000E066F000E076F5FEC1FF09A
:10314000CCEC1FF02AC182F40401300E82272FEC50
:103150000BF02BC182F40401300E82272FEC0BF010
:103160002CC182F40401300E82272FEC0BF02DC10C
:1031700082F40401300E82272FEC0BF02EC182F472
:103180000401300E82272FEC0BF02FC182F40401D2
:10319000300E82272FEC0BF030C182F40401300E88
:1031A00082272FEC0BF004012E0E826F2FEC0BF018
:1031B00031C182F40401300E82272FEC0BF032C1B2
:1031C00082F40401300E82272FEC0BF033C182F41D
:1031D0000401300E82272FEC0BF00401730E826F76
:1031E0002FEC0BF004012C0E826F2FEC0BF029EC6E
:1031F00020F059C100F15AC101F19FEC1AF088EC9E
:1032000012F00FB207EF19F00FA039EF19F0040117
:103210002C0E826F2FEC0BF0200EF86EF76AF66A18
:1032200004010900F5CF82F42FEC0BF00900F5CF73
:1032300082F42FEC0BF00900F5CF82F42FEC0BF0A9
:103240000900F5CF82F42FEC0BF00900F5CF82F4E2
:103250002FEC0BF00900F5CF82F42FEC0BF00900F6
:10326000F5CF82F42FEC0BF00900F5CF82F42FECB0
:103270000BF039EC0BF00F9075EF19F00401630EB1
:10328000826F2FEC0BF004012C0E826F2FEC0BF0F1
:103290007BEC19F004012C0E826F2FEC0BF0EEEC9E
:1032A00019F004012C0E826F2FEC0BF06AEC1AF06F
:1032B00004012C0E826F2FEC0BF00101F80E006F51
:1032C000CD0E016F660E026F030E036F90EC19F0C6
:1032D00004012C0E826F2FEC0BF080EC1AF039EC0D
:1032E0000BF075EF19F039EC0BF00301C26B07908E
:1032F000109284EF1CF0D8900E0E20EC09F0E8CF6D
:1033000000F10F0E20EC09F0E8CF01F1100E20ECD7
:1033100009F0E8CF02F1110E20EC09F0E8CF03F13B
:103320000101000E046F000E056F010E066F000E06
:10333000076F5FEC1FF0CCEC1FF02AC182F4040190
:10334000300E82272FEC0BF02BC182F40401300EDB
:1033500082272FEC0BF02CC182F40401300E82275F
:103360002FEC0BF02DC182F40401300E82272FECDC
:103370000BF02EC182F40401300E82272FEC0BF0EB
:103380002FC182F40401300E82272FEC0BF030C1E4
:1033900082F40401300E82272FEC0BF031C182F44D
:1033A0000401300E82272FEC0BF004012E0E826FE9
:1033B0002FEC0BF032C182F40401300E82272FEC87
:1033C0000BF033C182F40401300E82272FEC0BF096
:1033D00004016D0E826F2FEC0BF01200120E20EC28
:1033E00009F0E8CF00F1130E20EC09F0E8CF01F16D
:1033F000140E20EC09F0E8CF02F1150E20EC09F0D4
:10340000E8CF03F101010A0E046F000E056F000EF4
:10341000066F000E076F3FEC1FF0000E046F120ED8
:10342000056F000E066F000E076F5FEC1FF0CCEC0F
:103430001FF02AC182F40401300E82272FEC0BF01A
:103440002BC182F40401300E82272FEC0BF02CC12B
:1034500082F40401300E82272FEC0BF02DC182F490
:103460000401300E82272FEC0BF02EC182F40401F0
:10347000300E82272FEC0BF02FC182F40401300EA6
:1034800082272FEC0BF030C182F40401300E82272A
:103490002FEC0BF004012E0E826F2FEC0BF031C1DC
:1034A00082F40401300E82272FEC0BF032C182F43B
:1034B0000401300E82272FEC0BF033C182F404019B
:1034C000300E82272FEC0BF00401730E826F2FEC6D
:1034D0000BF012000A0E20EC09F0E8CF00F10B0E01
:1034E00020EC09F0E8CF01F10C0E20EC09F0E8CF58
:1034F00002F10D0E20EC09F0E8CF03F19FEF1AF076
:10350000060E20EC09F0E8CF00F1070E20EC09F0E0
:10351000E8CF01F1080E20EC09F0E8CF02F1090E26
:1035200020EC09F0E8CF03F19FEF1AF0010129EC3C
:1035300020F0078457C100F158C101F1079401013F
:10354000E80E046F800E056F000E066F000E076F09
:103550003FEC1FF0000E046F040E056F000E066FA7
:10356000000E076F5FEC1FF0880E046F130E056FDF
:10357000000E066F000E076F2EEC1FF00A0E046F90
:10358000000E056F000E066F000E076F5FEC1FF058
:10359000CCEC1FF001012967D3EF1AF00401200ED3
:1035A000826FD6EF1AF004012D0E826F2FEC0BF014
:1035B00030C182F40401300E82272FEC0BF031C1B0
:1035C00082F40401300E82272FEC0BF032C182F41A
:1035D0000401300E82272FEC0BF004012E0E826FB7
:1035E0002FEC0BF033C182F40401300E82272FEC54
:1035F0000BF00401430E826F2FEC0BF0120087C317
:103600002AF188C32BF189C32CF18AC32DF18BC316
:103610002EF18CC32FF18DC330F18EC331F190C3E5
:1036200032F191C333F10101296B77EC20F0EEEC1C
:103630001FF00101000E046F000E056F010E066FF2
:10364000000E076F3FEC1FF00E0E0C6E00C10BF06A
:1036500009EC09F00F0E0C6E01C10BF009EC09F03A
:10366000100E0C6E02C10BF009EC09F0110E0C6E7D
:1036700003C10BF009EC09F004017A0E826F2FEC04
:103680000BF004012C0E826F2FEC0BF00401350EB1
:10369000826F2FEC0BF004012C0E826F2FEC0BF0DD
:1036A0007BEC19F011EF14F087C32AF188C32BF1DA
:1036B00089C32CF18AC32DF18BC32EF18CC32FF15A
:1036C0008DC330F18EC331F190C332F191C333F128
:1036D0000101296B77EC20F0EEEC1FF0880E046FEF
:1036E000130E056F000E066F000E076F33EC1FF010
:1036F000000E046F040E056F000E066F000E076FBC
:103700003FEC1FF00101E80E046F800E056F000E04
:10371000066F000E076F5FEC1FF00A0E0C6E00C103
:103720000BF009EC09F00B0E0C6E01C10BF009EC6B
:1037300009F00C0E0C6E02C10BF009EC09F00D0E35
:103740000C6E03C10BF009EC09F004017A0E826FD4
:103750002FEC0BF004012C0E826F2FEC0BF0040108
:10376000360E826F2FEC0BF004012C0E826F2FECC3
:103770000BF06AEC1AF011EF14F087C32AF188C33A
:103780002BF189C32CF18AC32DF18BC32EF18CC38D
:103790002FF18DC330F18FC331F190C332F191C35A
:1037A00033F1010177EC20F0EEEC1FF0000E046F16
:1037B000120E056F000E066F000E076F3FEC1FF034
:1037C00001010A0E046F000E056F000E066F000E59
:1037D000076F5FEC1FF0120E0C6E00C10BF009ECCE
:1037E00009F0130E0C6E01C10BF009EC09F0140E78
:1037F0000C6E02C10BF009EC09F0150E0C6E03C142
:103800000BF009EC09F004017A0E826F2FEC0BF03B
:1038100004012C0E826F2FEC0BF00401370E826F27
:103820002FEC0BF004012C0E826F2FEC0BF0EEEC62
:1038300019F011EF14F087C32AF188C32BF189C363
:103840002CF18AC32DF18BC32EF18CC32FF18DC3C4
:1038500030F18EC331F190C332F191C333F10101E4
:10386000296B77EC20F0EEEC1FF0880E046F130E3E
:10387000056F000E066F000E076F33EC1FF0000E91
:10388000046F040E056F000E066F000E076F3FEC0D
:103890001FF00101E80E046F800E056F000E066F29
:1038A000000E076F5FEC1FF0060E0C6E00C10BF0F0
:1038B00009EC09F0070E0C6E01C10BF009EC09F0E0
:1038C000080E0C6E02C10BF009EC09F0090E0C6E2B
:1038D00003C10BF009EC09F004017A0E826F2FECA2
:1038E0000BF004012C0E826F2FEC0BF00401380E4C
:1038F000826F2FEC0BF004012C0E826F2FEC0BF07B
:1039000080EC1AF011EF14F007A8F7EF1CF001019A
:10391000800E006F1A0E016F060E026F000E036F0D
:103920004BC104F14CC105F14DC106F14EC107F187
:103930002EEC1FF003BF3DEF1DF089EC1DF04BC1D5
:1039400000F14CC101F14DC102F14EC103F10782FA
:103950003BEC1EF018C104F119C105F11AC106F1C2
:103960001BC107F1F80E006FCD0E016F660E026FDE
:10397000030E036F2EEC1FF00E0E0C6E00C10BF049
:1039800009EC09F00F0E0C6E01C10BF009EC09F007
:10399000100E0C6E02C10BF009EC09F0110E0C6E4A
:1039A00003C10BF009EC09F00784010129EC20F0B8
:1039B00057C100F158C101F107940A0E0C6E00C105
:1039C0000BF009EC09F00B0E0C6E01C10BF009ECC9
:1039D00009F00C0E0C6E02C10BF009EC09F00D0E93
:1039E0000C6E03C10BF009EC09F03DEF1DF007AAC6
:1039F0003DEF1DF00784010129EC20F057C100F1D3
:103A000058C101F10794060E0C6E00C10BF009ECD1
:103A100009F0070E0C6E01C10BF009EC09F0080E5D
:103A20000C6E02C10BF009EC09F0090E0C6E03C11B
:103A30000BF009EC09F0078462C100F163C101F1E8
:103A400064C102F165C103F10794120E0C6E00C14E
:103A50000BF009EC09F0130E0C6E01C10BF009EC30
:103A600009F0140E0C6E02C10BF009EC09F0150EF2
:103A70000C6E03C10BF009EC09F00798079A0401DA
:103A8000805181197F0B0DE09EA8FED714EE00F047
:103A900081517F0BE126E750812B0F01AD6E3FEF87
:103AA0001DF081EF0AF018C100F119C101F11AC12E
:103AB00002F11BC103F1000E046F000E056F010E31
:103AC000066F000E076F5FEC1FF029A17EEF1DF05F
:103AD0002051D8B47EEF1DF018C100F119C101F1D9
:103AE0001AC102F11BC103F1000E046F000E056F35
:103AF0000A0E066F000E076F5FEC1FF01200010147
:103B00000451001305510113065102130751031309
:103B100012000101186B196B1A6B1B6B12002AC182
:103B200082F40401300E82272FEC0BF02BC182F4BB
:103B30000401300E82272FEC0BF02CC182F404011B
:103B4000300E82272FEC0BF02DC182F40401300ED1
:103B500082272FEC0BF02EC182F40401300E822755
:103B60002FEC0BF02FC182F40401300E82272FECD2
:103B70000BF030C182F40401300E82272FEC0BF0E1
:103B800031C182F40401300E82272FEC0BF032C1D8
:103B900082F40401300E82272FEC0BF033C182F443
:103BA0000401300E82272FEC0BF012002FC182F49B
:103BB0000401300E82272FEC0BF030C182F4040197
:103BC000300E82272FEC0BF031C182F40401300E4D
:103BD00082272FEC0BF032C182F40401300E8227D1
:103BE0002FEC0BF033C182F40401300E82272FEC4E
:103BF0000BF01200060E1E6E060E1F6E060E206ED5
:103C00001E2E00EF1EF01F2E00EF1EF0202E00EFE4
:103C10001EF08B84020E1E6E020E1F6E020E206EB0
:103C20001E2E10EF1EF01F2E10EF1EF0202E10EF94
:103C30001EF08B941200FF0E1F6E1FC020F0030EAB
:103C40001E6E8B841E2E21EF1EF0030E1E6E202E84
:103C500021EF1EF08B941FC020F0030E1E6E1E2E4F
:103C60002FEF1EF0030E1E6E203E2FEF1EF01F2EB4
:103C70001DEF1EF012000101005305E1015303E1A5
:103C8000025301E1002BFEEC1EF029EC20F039512B
:103C9000006F3A51016F420E046F4B0E056F000E1C
:103CA000066F000E076F3FEC1FF000C104F101C169
:103CB00005F102C106F103C107F118C100F119C1F4
:103CC00001F11AC102F11BC103F107B26CEF1EF042
:103CD00033EC1FF06EEF1EF02EEC1FF000C118F158
:103CE00001C119F102C11AF103C11BF1120029EC43
:103CF00020F059C100F15AC101F1060E20EC09F083
:103D0000E8CF04F1070E20EC09F0E8CF05F1080E2A
:103D100020EC09F0E8CF06F1090E20EC09F0E8CF1D
:103D200007F12EEC1FF000C124F101C125F102C101
:103D300026F103C127F1290E046F000E056F000E56
:103D4000066F000E076F3FEC1FF0EE0E046F430E80
:103D5000056F000E066F000E076F33EC1FF024C1D5
:103D600004F125C105F126C106F127C107F13FEC99
:103D70001FF000C11CF101C11DF102C11EF103C100
:103D80001FF1120E20EC09F0E8CF04F1130E20EC25
:103D900009F0E8CF05F1140E20EC09F0E8CF06F1A8
:103DA000150E20EC09F0E8CF07F10D0E006F000EA4
:103DB000016F000E026F000E036F3FEC1FF0180E34
:103DC000046F000E056F000E066F000E076F5FECAC
:103DD0001FF01CC104F11DC105F11EC106F11FC178
:103DE00007F133EC1FF06A0E046F2A0E056F000E08
:103DF000066F000E076F2EEC1FF01200BF0EFA6E5A
:103E0000200E3A6F396BD8900037013702370337ED
:103E1000D8B00FEF1FF03A2F04EF1FF039073A0721
:103E20000353D8B412000331070B80093F6F0339E5
:103E30000F0B010F396F80EC5FF0406F390580EC9C
:103E40005FF0405D405F396B3F33D8B0392739337D
:103E50003FA924EF1FF040513927120001014EEC19
:103E600020F0D8B01200010103510719346F11EC92
:103E700020F0D8900751031934AF800F12000101D0
:103E8000346B35EC20F0D8A04BEC20F0D8B0120009
:103E900020EC20F029EC20F01F0E366F61EC20F0B2
:103EA0000B35D8B011EC20F0D8A00335D8B01200F3
:103EB000362F4EEF1FF034B138EC20F01200010124
:103EC000346B04510511061107110008D8A035EC18
:103ED00020F0D8A04BEC20F0D8B01200086B096B92
:103EE0000A6B0B6B61EC20F01F0E366F61EC20F05B
:103EF00007510B5DD8A489EF1FF006510A5DD8A4C5
:103F000089EF1FF00551095DD8A489EF1FF0045116
:103F1000085DD8A09CEF1FF00451085F0551D8A0A0
:103F2000053D095F0651D8A0063D0A5F0751D8A09C
:103F3000073D0B5FD8900081362F76EF1FF034B12C
:103F400038EC20F0346B35EC20F0D89065EC20F0A4
:103F500007510B5DD8A4B9EF1FF006510A5DD8A434
:103F6000B9EF1FF00551095DD8A4B9EF1FF0045156
:103F7000085DD8A0C8EF1FF0003FC8EF1FF0013F59
:103F8000C8EF1FF0023FC8EF1FF0032BD8B4120098
:103F900034B138EC20F012000101346B35EC20F024
:103FA000D8B012006AEC20F0200E366F00370137CF
:103FB0000237033711EE33F00A0E376FE7360A0E79
:103FC000E75CD8B0E76EE552372FDEEF1FF0362FF3
:103FD000D6EF1FF034B12981D890120001010A0EEA
:103FE000346F200E366F11EE29F03451376F0A0E00
:103FF000D890E652D8B0E726E732372FF9EF1FF016
:104000000333023301330033362FF3EF1FF0E75051
:10401000FF0FD8A00335D8B0120029B138EC20F03A
:104020001200045100270551D8B0053D0127065163
:10403000D8B0063D02270751D8B0073D032712002C
:104040000051086F0151096F02510A6F03510B6F44
:1040500012000101006B016B026B036B1200010186
:10406000046B056B066B076B12000335D8A01200BA
:104070000351800B001F011F021F031F003F48EF69
:1040800020F0013F48EF20F0023F48EF20F0032BE3
:10409000342B032512000735D8A012000751800BDE
:1040A000041F051F061F071F043F5EEF20F0053F9A
:1040B0005EEF20F0063F5EEF20F0072B342B072544
:1040C00012000037013702370337083709370A373C
:1040D0000B3712000101296B2A6B2B6B2C6B2D6B9C
:1040E0002E6B2F6B306B316B326B336B1200010117
:1040F0002A510F0B2A6F2B510F0B2B6F2C510F0BCB
:104100002C6F2D510F0B2D6F2E510F0B2E6F2F512A
:104110000F0B2F6F30510F0B306F31510F0B316F71
:0E41200032510F0B326F33510F0B336F120001
:10BF0000E844F926000C160C2B0C3F0C520C640C68
:10BF1000760C860C960CA50CB30CC10CCF0CDC0C6B
:06BF2000E80CF40C000C1B
:00000001FF
